
 Start         Length     Name                   Class
 0001:00401000 000039B8H .text                   CODE
 0002:00405000 00000284H .itext                  ICODE
 0003:00406000 00000078H .data                   DATA
 0004:00407000 00000020H .bss                    BSS
 0005:00000000 00000000H .tls                    TLS


Detailed map of segments

 0001:00000000 00000136 C=CODE     S=.text    G=(none)   M=System   ACBP=A9
 0001:00000138 000001C3 C=CODE     S=.text    G=(none)   M=SysInit  ACBP=A9
 0001:000002FC 00000071 C=CODE     S=.text    G=(none)   M=Windows  ACBP=A9
 0001:00000370 0000002E C=CODE     S=.text    G=(none)   M=SysUtils ACBP=A9
 0001:000003A0 000000A6 C=CODE     S=.text    G=(none)   M=Classes  ACBP=A9
 0001:00000448 0000000E C=CODE     S=.text    G=(none)   M=TypInfo  ACBP=A9
 0001:00000458 00000006 C=CODE     S=.text    G=(none)   M=Variants ACBP=A9
 0001:00000460 00000006 C=CODE     S=.text    G=(none)   M=VarUtils ACBP=A9
 0001:00000468 00000006 C=CODE     S=.text    G=(none)   M=DesignIntf ACBP=A9
 0001:00000470 000002CE C=CODE     S=.text    G=(none)   M=Controls ACBP=A9
 0001:00000740 00000006 C=CODE     S=.text    G=(none)   M=SyncObjs ACBP=A9
 0001:00000748 00000006 C=CODE     S=.text    G=(none)   M=TimeSpan ACBP=A9
 0001:00000750 00000006 C=CODE     S=.text    G=(none)   M=ActnList ACBP=A9
 0001:00000758 0000001E C=CODE     S=.text    G=(none)   M=Graphics ACBP=A9
 0001:00000778 00000006 C=CODE     S=.text    G=(none)   M=Registry ACBP=A9
 0001:00000780 00000006 C=CODE     S=.text    G=(none)   M=IniFiles ACBP=A9
 0001:00000788 0000000E C=CODE     S=.text    G=(none)   M=IOUtils  ACBP=A9
 0001:00000798 00000006 C=CODE     S=.text    G=(none)   M=Themes   ACBP=A9
 0001:000007A0 00000006 C=CODE     S=.text    G=(none)   M=Menus    ACBP=A9
 0001:000007A8 00000006 C=CODE     S=.text    G=(none)   M=UxTheme  ACBP=A9
 0001:000007B0 00000006 C=CODE     S=.text    G=(none)   M=MultiMon ACBP=A9
 0001:000007B8 0000006E C=CODE     S=.text    G=(none)   M=Forms    ACBP=A9
 0001:00000828 00000006 C=CODE     S=.text    G=(none)   M=HelpIntfs ACBP=A9
 0001:00000830 00000006 C=CODE     S=.text    G=(none)   M=Dialogs  ACBP=A9
 0001:00000838 00000006 C=CODE     S=.text    G=(none)   M=ComCtrls ACBP=A9
 0001:00000840 00000006 C=CODE     S=.text    G=(none)   M=GraphUtil ACBP=A9
 0001:00000848 0000001E C=CODE     S=.text    G=(none)   M=StdCtrls ACBP=A9
 0001:00000868 00000066 C=CODE     S=.text    G=(none)   M=ExtCtrls ACBP=A9
 0001:000008D0 00000006 C=CODE     S=.text    G=(none)   M=Printers ACBP=A9
 0001:000008D8 00000006 C=CODE     S=.text    G=(none)   M=Clipbrd  ACBP=A9
 0001:000008E0 00000006 C=CODE     S=.text    G=(none)   M=FlatSB   ACBP=A9
 0001:000008E8 000023AF C=CODE     S=.text    G=(none)   M=Boxes    ACBP=A9
 0001:00002C98 0000000E C=CODE     S=.text    G=(none)   M=VCLEditors ACBP=A9
 0001:00002CA8 00000006 C=CODE     S=.text    G=(none)   M=DesignEditors ACBP=A9
 0001:00002CB0 00000006 C=CODE     S=.text    G=(none)   M=ToolsAPI ACBP=A9
 0001:00002CB8 00000006 C=CODE     S=.text    G=(none)   M=XMLIntf  ACBP=A9
 0001:00002CC0 00000006 C=CODE     S=.text    G=(none)   M=xmldom   ACBP=A9
 0001:00002CC8 00000006 C=CODE     S=.text    G=(none)   M=msxmldom ACBP=A9
 0001:00002CD0 00000006 C=CODE     S=.text    G=(none)   M=ComObj   ACBP=A9
 0001:00002CD8 00000006 C=CODE     S=.text    G=(none)   M=DockForm ACBP=A9
 0001:00002CE0 00000006 C=CODE     S=.text    G=(none)   M=IDEMessages ACBP=A9
 0001:00002CE8 00000006 C=CODE     S=.text    G=(none)   M=DeskForm ACBP=A9
 0001:00002CF0 00000006 C=CODE     S=.text    G=(none)   M=BaseDock ACBP=A9
 0001:00002CF8 00000006 C=CODE     S=.text    G=(none)   M=PercentageDockTree ACBP=A9
 0001:00002D00 00000006 C=CODE     S=.text    G=(none)   M=CaptionedDockTree ACBP=A9
 0001:00002D08 00000006 C=CODE     S=.text    G=(none)   M=DockTabSet ACBP=A9
 0001:00002D10 00000006 C=CODE     S=.text    G=(none)   M=Tabs     ACBP=A9
 0001:00002D18 00000006 C=CODE     S=.text    G=(none)   M=DeskUtil ACBP=A9
 0001:00002D20 00000006 C=CODE     S=.text    G=(none)   M=TabDock  ACBP=A9
 0001:00002D28 00000006 C=CODE     S=.text    G=(none)   M=PlatformDefaultStyleActnCtrls ACBP=A9
 0001:00002D30 00000006 C=CODE     S=.text    G=(none)   M=Buttons  ACBP=A9
 0001:00002D38 00000006 C=CODE     S=.text    G=(none)   M=ActnMan  ACBP=A9
 0001:00002D40 00000006 C=CODE     S=.text    G=(none)   M=ActnMenus ACBP=A9
 0001:00002D48 00000006 C=CODE     S=.text    G=(none)   M=ExtActns ACBP=A9
 0001:00002D50 00000006 C=CODE     S=.text    G=(none)   M=ExtDlgs  ACBP=A9
 0001:00002D58 00000006 C=CODE     S=.text    G=(none)   M=Mapi     ACBP=A9
 0001:00002D60 00000006 C=CODE     S=.text    G=(none)   M=Proxies  ACBP=A9
 0001:00002D68 00000006 C=CODE     S=.text    G=(none)   M=ComponentDesigner ACBP=A9
 0001:00002D70 00000006 C=CODE     S=.text    G=(none)   M=IDEHelp  ACBP=A9
 0001:00002D78 00000006 C=CODE     S=.text    G=(none)   M=AxCtrls  ACBP=A9
 0001:00002D80 00000006 C=CODE     S=.text    G=(none)   M=StFilSys ACBP=A9
 0001:00002D88 00000006 C=CODE     S=.text    G=(none)   M=WideStrings ACBP=A9
 0001:00002D90 00000006 C=CODE     S=.text    G=(none)   M=TopLevels ACBP=A9
 0001:00002D98 00000006 C=CODE     S=.text    G=(none)   M=TreeIntf ACBP=A9
 0001:00002DA0 00000006 C=CODE     S=.text    G=(none)   M=AppEvnts ACBP=A9
 0001:00002DA8 0000048F C=CODE     S=.text    G=(none)   M=ccreg    ACBP=A9
 0001:00003238 0000025E C=CODE     S=.text    G=(none)   M=ccregprc ACBP=A9
 0001:00003498 0000051F C=CODE     S=.text    G=(none)   M=.ccpackD2010 ACBP=A9
 0002:00000000 00000006 C=ICODE    S=.itext   G=(none)   M=System   ACBP=A9
 0002:00000008 00000016 C=ICODE    S=.itext   G=(none)   M=Windows  ACBP=A9
 0002:00000020 0000001E C=ICODE    S=.itext   G=(none)   M=SysUtils ACBP=A9
 0002:00000040 0000000E C=ICODE    S=.itext   G=(none)   M=Classes  ACBP=A9
 0002:00000050 00000006 C=ICODE    S=.itext   G=(none)   M=TypInfo  ACBP=A9
 0002:00000058 00000006 C=ICODE    S=.itext   G=(none)   M=Variants ACBP=A9
 0002:00000060 00000006 C=ICODE    S=.itext   G=(none)   M=VarUtils ACBP=A9
 0002:00000068 00000006 C=ICODE    S=.itext   G=(none)   M=Controls ACBP=A9
 0002:00000070 00000006 C=ICODE    S=.itext   G=(none)   M=SyncObjs ACBP=A9
 0002:00000078 00000006 C=ICODE    S=.itext   G=(none)   M=TimeSpan ACBP=A9
 0002:00000080 00000006 C=ICODE    S=.itext   G=(none)   M=ActnList ACBP=A9
 0002:00000088 00000006 C=ICODE    S=.itext   G=(none)   M=Graphics ACBP=A9
 0002:00000090 00000006 C=ICODE    S=.itext   G=(none)   M=Registry ACBP=A9
 0002:00000098 00000006 C=ICODE    S=.itext   G=(none)   M=IniFiles ACBP=A9
 0002:000000A0 0000000E C=ICODE    S=.itext   G=(none)   M=IOUtils  ACBP=A9
 0002:000000B0 00000006 C=ICODE    S=.itext   G=(none)   M=Themes   ACBP=A9
 0002:000000B8 00000006 C=ICODE    S=.itext   G=(none)   M=Menus    ACBP=A9
 0002:000000C0 00000006 C=ICODE    S=.itext   G=(none)   M=UxTheme  ACBP=A9
 0002:000000C8 00000006 C=ICODE    S=.itext   G=(none)   M=MultiMon ACBP=A9
 0002:000000D0 00000006 C=ICODE    S=.itext   G=(none)   M=Forms    ACBP=A9
 0002:000000D8 00000006 C=ICODE    S=.itext   G=(none)   M=HelpIntfs ACBP=A9
 0002:000000E0 00000006 C=ICODE    S=.itext   G=(none)   M=Dialogs  ACBP=A9
 0002:000000E8 00000006 C=ICODE    S=.itext   G=(none)   M=ComCtrls ACBP=A9
 0002:000000F0 00000006 C=ICODE    S=.itext   G=(none)   M=GraphUtil ACBP=A9
 0002:000000F8 00000006 C=ICODE    S=.itext   G=(none)   M=ExtCtrls ACBP=A9
 0002:00000100 00000006 C=ICODE    S=.itext   G=(none)   M=Printers ACBP=A9
 0002:00000108 00000006 C=ICODE    S=.itext   G=(none)   M=Clipbrd  ACBP=A9
 0002:00000110 00000006 C=ICODE    S=.itext   G=(none)   M=FlatSB   ACBP=A9
 0002:00000118 00000008 C=ICODE    S=.itext   G=(none)   M=Boxes    ACBP=A9
 0002:00000120 0000000E C=ICODE    S=.itext   G=(none)   M=VCLEditors ACBP=A9
 0002:00000130 00000006 C=ICODE    S=.itext   G=(none)   M=DesignEditors ACBP=A9
 0002:00000138 00000006 C=ICODE    S=.itext   G=(none)   M=ToolsAPI ACBP=A9
 0002:00000140 00000006 C=ICODE    S=.itext   G=(none)   M=XMLIntf  ACBP=A9
 0002:00000148 00000006 C=ICODE    S=.itext   G=(none)   M=xmldom   ACBP=A9
 0002:00000150 00000006 C=ICODE    S=.itext   G=(none)   M=msxmldom ACBP=A9
 0002:00000158 00000006 C=ICODE    S=.itext   G=(none)   M=ComObj   ACBP=A9
 0002:00000160 00000006 C=ICODE    S=.itext   G=(none)   M=DockForm ACBP=A9
 0002:00000168 00000006 C=ICODE    S=.itext   G=(none)   M=IDEMessages ACBP=A9
 0002:00000170 00000006 C=ICODE    S=.itext   G=(none)   M=DeskForm ACBP=A9
 0002:00000178 00000006 C=ICODE    S=.itext   G=(none)   M=BaseDock ACBP=A9
 0002:00000180 00000006 C=ICODE    S=.itext   G=(none)   M=PercentageDockTree ACBP=A9
 0002:00000188 00000006 C=ICODE    S=.itext   G=(none)   M=CaptionedDockTree ACBP=A9
 0002:00000190 00000006 C=ICODE    S=.itext   G=(none)   M=DockTabSet ACBP=A9
 0002:00000198 00000006 C=ICODE    S=.itext   G=(none)   M=Tabs     ACBP=A9
 0002:000001A0 00000006 C=ICODE    S=.itext   G=(none)   M=DeskUtil ACBP=A9
 0002:000001A8 00000006 C=ICODE    S=.itext   G=(none)   M=TabDock  ACBP=A9
 0002:000001B0 00000006 C=ICODE    S=.itext   G=(none)   M=PlatformDefaultStyleActnCtrls ACBP=A9
 0002:000001B8 00000006 C=ICODE    S=.itext   G=(none)   M=Buttons  ACBP=A9
 0002:000001C0 00000006 C=ICODE    S=.itext   G=(none)   M=ActnMan  ACBP=A9
 0002:000001C8 00000006 C=ICODE    S=.itext   G=(none)   M=ActnMenus ACBP=A9
 0002:000001D0 00000006 C=ICODE    S=.itext   G=(none)   M=ExtActns ACBP=A9
 0002:000001D8 00000006 C=ICODE    S=.itext   G=(none)   M=ExtDlgs  ACBP=A9
 0002:000001E0 00000006 C=ICODE    S=.itext   G=(none)   M=Mapi     ACBP=A9
 0002:000001E8 00000006 C=ICODE    S=.itext   G=(none)   M=Proxies  ACBP=A9
 0002:000001F0 00000006 C=ICODE    S=.itext   G=(none)   M=ComponentDesigner ACBP=A9
 0002:000001F8 00000006 C=ICODE    S=.itext   G=(none)   M=IDEHelp  ACBP=A9
 0002:00000200 00000006 C=ICODE    S=.itext   G=(none)   M=AxCtrls  ACBP=A9
 0002:00000208 00000006 C=ICODE    S=.itext   G=(none)   M=StFilSys ACBP=A9
 0002:00000210 00000006 C=ICODE    S=.itext   G=(none)   M=WideStrings ACBP=A9
 0002:00000218 00000006 C=ICODE    S=.itext   G=(none)   M=TopLevels ACBP=A9
 0002:00000220 00000006 C=ICODE    S=.itext   G=(none)   M=TreeIntf ACBP=A9
 0002:00000228 00000006 C=ICODE    S=.itext   G=(none)   M=AppEvnts ACBP=A9
 0002:00000230 0000002F C=ICODE    S=.itext   G=(none)   M=ccreg    ACBP=A9
 0002:00000260 0000001A C=ICODE    S=.itext   G=(none)   M=ccregprc ACBP=A9
 0002:0000027C 00000005 C=ICODE    S=.itext   G=(none)   M=.ccpackD2010 ACBP=A9
 0003:00000000 00000030 C=DATA     S=.data    G=DGROUP   M=SysInit  ACBP=A9
 0003:00000030 0000000C C=DATA     S=.data    G=DGROUP   M=Windows  ACBP=A9
 0003:0000003C 00000020 C=DATA     S=.data    G=DGROUP   M=ccreg    ACBP=A9
 0004:00000000 0000000C C=BSS      S=.bss     G=DGROUP   M=SysInit  ACBP=A9
 0004:0000000C 00000008 C=BSS      S=.bss     G=DGROUP   M=Windows  ACBP=A9
 0004:00000014 00000004 C=BSS      S=.bss     G=DGROUP   M=Boxes    ACBP=A9
 0004:00000018 00000004 C=BSS      S=.bss     G=DGROUP   M=ccreg    ACBP=A9
 0004:0000001C 00000004 C=BSS      S=.bss     G=DGROUP   M=ccregprc ACBP=A9


  Address             Publics by Name

 0002:0000027C       .ccpackD2010..ccpackD2010
 0001:00003998       .ccpackD2010.@GetPackageInfoTable
 0001:000039A0       .ccpackD2010.@PackageLoad
 0001:000039AC       .ccpackD2010.@PackageUnload
 0002:00000080       ActnList.ActnList
 0001:00000750       ActnList.Finalization
 0002:000001C0       ActnMan.ActnMan
 0001:00002D38       ActnMan.Finalization
 0002:000001C8       ActnMenus.ActnMenus
 0001:00002D40       ActnMenus.Finalization
 0002:00000228       AppEvnts.AppEvnts
 0001:00002DA0       AppEvnts.Finalization
 0002:00000200       AxCtrls.AxCtrls
 0001:00002D78       AxCtrls.Finalization
 0002:00000178       BaseDock.BaseDock
 0001:00002CF0       BaseDock.Finalization
 0004:00000014       Boxes..4
 0001:000008E8       Boxes..TBox
 0001:000014C0       Boxes..TControlGroupBox
 0001:00001F20       Boxes..TControlScrollBox
 0001:00002408       Boxes.AdjustColors
 0002:00000118       Boxes.Boxes
 0001:00002C90       Boxes.Finalization
 0001:000021C0       Boxes.TBox.Create
 0001:000023B0       Boxes.TBox.CreateParams
 0001:00002328       Boxes.TBox.Destroy
 0001:00002500       Boxes.TBox.GetChildren
 0001:00002440       Boxes.TBox.Paint
 0001:0000256C       Boxes.TBox.SetChildOrder
 0001:000023D8       Boxes.TBox.SetParent
 0001:00002600       Boxes.TControlGroupBox.Create
 0001:000027F0       Boxes.TControlGroupBox.CreateParams
 0001:00002768       Boxes.TControlGroupBox.Destroy
 0001:00002848       Boxes.TControlGroupBox.GetChildren
 0001:000028B4       Boxes.TControlGroupBox.SetChildOrder
 0001:00002818       Boxes.TControlGroupBox.SetParent
 0001:00002948       Boxes.TControlScrollBox.Create
 0001:00002B38       Boxes.TControlScrollBox.CreateParams
 0001:00002AB0       Boxes.TControlScrollBox.Destroy
 0001:00002B90       Boxes.TControlScrollBox.GetChildren
 0001:00002BFC       Boxes.TControlScrollBox.SetChildOrder
 0001:00002B60       Boxes.TControlScrollBox.SetParent
 0002:000001B8       Buttons.Buttons
 0001:00002D30       Buttons.Finalization
 0002:00000188       CaptionedDockTree.CaptionedDockTree
 0001:00002D00       CaptionedDockTree.Finalization
 0004:00000018       ccreg..1
 0003:00000040       ccreg.BaseContainerClassArray
 0002:00000230       ccreg.ccreg
 0001:00002E3C       ccreg.ClassNotFound
 0003:00000058       ccreg.CustomContainerClassList
 0001:00003210       ccreg.Finalization
 0001:00002F30       ccreg.FindCustomContainerClass
 0001:00002E08       ccreg.GetBaseContainer
 0001:00002EA8       ccreg.GetCustomContainerClass
 0001:00002F74       ccreg.GetCustomContainerClass
 0001:00002FCC       ccreg.GetCustomContainerClassListCount
 0001:00002F50       ccreg.GetCustomContainerUnit
 0001:00002DE8       ccreg.IsBaseContainer
 0001:000031BC       ccreg.ModuleUnload
 0001:00003014       ccreg.RegisterCustomContainer
 0003:0000003C       ccreg.RegisterCustomContainerProc
 0001:00003128       ccreg.UnRegisterCustomContainer
 0001:00003138       ccreg.UnRegisterCustomContainerClasses
 0004:0000001C       ccregprc..1
 0002:00000260       ccregprc.ccregprc
 0001:00003484       ccregprc.Finalization
 0001:00003464       ccregprc.InitBaseContainerList
 0001:00003238       ccregprc.RegisterCustomContainerProcImpl
 0002:00000048       Classes.Classes
 0001:00000440       Classes.Finalization
 0001:000003A0       Classes.InitInheritedComponent
 0001:000003F0       Classes.TComponent.BeforeDestruction
 0001:00000408       Classes.TComponent.GetComponent
 0001:00000410       Classes.TComponent.GetComponentCount
 0001:00000438       Classes.TComponent.QueryInterface
 0001:00000428       Classes.TComponent.SafeCallException
 0001:00000418       Classes.TComponent.SetComponentIndex
 0001:00000420       Classes.TComponent.UpdateAction
 0001:00000430       Classes.TComponent.UpdateRegistry
 0001:00000400       Classes.TComponent.ValidateRename
 0001:000003F8       Classes.TComponent.WriteState
 0001:000003A8       Classes.TList.Add
 0001:000003B0       Classes.TList.Delete
 0001:000003B8       Classes.TList.Get
 0001:000003E0       Classes.TPersistent.Assign
 0002:00000040       Classes.TThread.Create@
 0001:000003E8       Classes.TThread.Destroy@
 0001:000003C0       Classes.TThreadList.Create
 0001:000003C8       Classes.TThreadList.LockList
 0001:000003D0       Classes.TThreadList.Remove
 0001:000003D8       Classes.TThreadList.UnlockList
 0002:00000108       Clipbrd.Clipbrd
 0001:000008D8       Clipbrd.Finalization
 0002:000000E8       ComCtrls.ComCtrls
 0001:00000838       ComCtrls.Finalization
 0002:00000158       ComObj.ComObj
 0001:00002CD0       ComObj.Finalization
 0002:000001F0       ComponentDesigner.ComponentDesigner
 0001:00002D68       ComponentDesigner.Finalization
 0002:00000068       Controls.Controls
 0001:00000738       Controls.Finalization
 0001:00000568       Controls.TControl.CreateTouchManager
 0001:00000558       Controls.TControl.DoGesture
 0001:00000560       Controls.TControl.DoGetGestureOptions
 0001:00000480       Controls.TControl.GetAction
 0001:00000470       Controls.TControl.GetDragImages
 0001:000004A0       Controls.TControl.GetDragMode
 0001:00000478       Controls.TControl.GetEnabled
 0001:00000598       Controls.TControl.GetFloating
 0001:000005A0       Controls.TControl.GetFloatingDockSiteClass
 0001:000004E8       Controls.TControl.GetText
 0001:000005A8       Controls.TControl.InitiateAction
 0001:00000490       Controls.TControl.IsAnchorsStored
 0001:00000518       Controls.TControl.IsBiDiModeStored
 0001:00000570       Controls.TControl.IsCaptionStored
 0001:00000540       Controls.TControl.IsColorStored
 0001:00000578       Controls.TControl.IsEnabledStored
 0001:00000508       Controls.TControl.IsFontStored
 0001:00000588       Controls.TControl.IsOnClickStored
 0001:00000510       Controls.TControl.IsShowHintStored
 0001:00000580       Controls.TControl.IsVisibleStored
 0001:00000590       Controls.TControl.Loaded
 0001:000004A8       Controls.TControl.SetAlign
 0001:00000488       Controls.TControl.SetAnchors
 0001:000004C0       Controls.TControl.SetAutoSize
 0001:000004F8       Controls.TControl.SetBiDiMode
 0001:00000538       Controls.TControl.SetColor
 0001:000005B0       Controls.TControl.SetConstraints
 0001:00000498       Controls.TControl.SetDragMode
 0001:000004D8       Controls.TControl.SetEnabled
 0001:00000500       Controls.TControl.SetFont
 0001:000004B8       Controls.TControl.SetHeight
 0001:000004C8       Controls.TControl.SetName
 0001:00000550       Controls.TControl.SetParentBiDiMode
 0001:00000548       Controls.TControl.SetParentColor
 0001:00000520       Controls.TControl.SetParentFont
 0001:00000530       Controls.TControl.SetParentShowHint
 0001:000004E0       Controls.TControl.SetPopupMenu
 0001:00000528       Controls.TControl.SetShowHint
 0001:000004F0       Controls.TControl.SetText
 0001:000004D0       Controls.TControl.SetVisible
 0001:000004B0       Controls.TControl.SetWidth
 0001:00000728       Controls.TCustomControl.Destroy
 0001:00000730       Controls.TCustomControl.PaintWindow
 0001:000005C0       Controls.TWinControl.AlignControls
 0001:000006F8       Controls.TWinControl.AssignTo
 0001:00000700       Controls.TWinControl.CanAutoSize
 0001:000006E8       Controls.TWinControl.CanResize
 0001:000006F0       Controls.TWinControl.ConstrainedResize
 0001:00000600       Controls.TWinControl.CreateHandle
 0001:000005E0       Controls.TWinControl.CreateWindowHandle
 0001:000005D8       Controls.TWinControl.CreateWnd
 0001:00000608       Controls.TWinControl.CustomAlignInsertBefore
 0001:00000610       Controls.TWinControl.CustomAlignPosition
 0001:00000630       Controls.TWinControl.DefaultHandler
 0001:000005E8       Controls.TWinControl.DefineProperties
 0001:00000618       Controls.TWinControl.DestroyHandle
 0001:000005F8       Controls.TWinControl.DestroyWindowHandle
 0001:000005F0       Controls.TWinControl.DestroyWnd
 0001:00000710       Controls.TWinControl.DockReplaceDockClient
 0001:000006D8       Controls.TWinControl.GetChildren
 0001:00000688       Controls.TWinControl.GetClientOrigin
 0001:00000690       Controls.TWinControl.GetClientRect
 0001:000005C8       Controls.TWinControl.GetControlCount
 0001:00000680       Controls.TWinControl.GetControlExtents
 0001:00000658       Controls.TWinControl.GetDeviceContext
 0001:000006B0       Controls.TWinControl.GetTabOrder
 0001:000006D0       Controls.TWinControl.HandleAllocated
 0001:00000660       Controls.TWinControl.Invalidate
 0001:000006A0       Controls.TWinControl.IsCtl3DStored
 0001:000005D0       Controls.TWinControl.Notification
 0001:000005B8       Controls.TWinControl.ReadState
 0001:00000670       Controls.TWinControl.Repaint
 0001:00000638       Controls.TWinControl.RequestAlign
 0001:00000648       Controls.TWinControl.SetBounds
 0001:000006E0       Controls.TWinControl.SetChildOrder
 0001:00000698       Controls.TWinControl.SetCtl3D
 0001:00000640       Controls.TWinControl.SetDockSite
 0001:00000678       Controls.TWinControl.SetFocus
 0001:00000720       Controls.TWinControl.SetParent
 0001:00000708       Controls.TWinControl.SetParentBackground
 0001:000006A8       Controls.TWinControl.SetParentCtl3D
 0001:00000620       Controls.TWinControl.SetParentDoubleBuffered
 0001:000006B8       Controls.TWinControl.SetTabOrder
 0001:000006C0       Controls.TWinControl.SetTabStop
 0001:000006C8       Controls.TWinControl.SetUseDockManager
 0001:00000650       Controls.TWinControl.ShowControl
 0001:00000668       Controls.TWinControl.Update
 0001:00000718       Controls.TWinControl.UpdateControlOriginalParentSize
 0001:00000628       Controls.TWinControl.WndProc
 0002:00000130       DesignEditors.DesignEditors
 0001:00002CA8       DesignEditors.Finalization
 0001:00000468       DesignIntf.RegisterCustomModule
 0002:00000170       DeskForm.DeskForm
 0001:00002CE8       DeskForm.Finalization
 0002:000001A0       DeskUtil.DeskUtil
 0001:00002D18       DeskUtil.Finalization
 0002:000000E0       Dialogs.Dialogs
 0001:00000830       Dialogs.Finalization
 0002:00000160       DockForm.DockForm
 0001:00002CD8       DockForm.Finalization
 0002:00000190       DockTabSet.DockTabSet
 0001:00002D08       DockTabSet.Finalization
 0002:000001D0       ExtActns.ExtActns
 0001:00002D48       ExtActns.Finalization
 0002:000000F8       ExtCtrls.ExtCtrls
 0001:000008C8       ExtCtrls.Finalization
 0001:00000868       ExtCtrls.Frame3D
 0001:000008B0       ExtCtrls.TCustomPanel.AdjustClientRect
 0001:000008B8       ExtCtrls.TCustomPanel.CanAutoSize
 0001:00000870       ExtCtrls.TCustomPanel.Create
 0001:00000878       ExtCtrls.TCustomPanel.CreateParams
 0001:00000880       ExtCtrls.TCustomPanel.SetAlignment
 0001:00000888       ExtCtrls.TCustomPanel.SetBevelInner
 0001:00000890       ExtCtrls.TCustomPanel.SetBevelOuter
 0001:00000898       ExtCtrls.TCustomPanel.SetBevelWidth
 0001:000008A8       ExtCtrls.TCustomPanel.SetBorderStyle
 0001:000008A0       ExtCtrls.TCustomPanel.SetBorderWidth
 0001:000008C0       ExtCtrls.TCustomPanel.SetParentBackground
 0002:000001D8       ExtDlgs.ExtDlgs
 0001:00002D50       ExtDlgs.Finalization
 0001:000008E0       FlatSB.Finalization
 0002:00000110       FlatSB.FlatSB
 0001:00000820       Forms.Finalization
 0002:000000D0       Forms.Forms
 0001:00000818       Forms.TApplication.HandleException
 0001:00000800       Forms.TScrollBox.Create
 0001:00000808       Forms.TScrollBox.CreateParams
 0001:00000810       Forms.TScrollBox.PaintWindow
 0001:000007F8       Forms.TScrollingWinControl.AdjustClientRect
 0001:000007C8       Forms.TScrollingWinControl.AlignControls
 0001:000007D0       Forms.TScrollingWinControl.AutoScrollEnabled
 0001:000007E8       Forms.TScrollingWinControl.AutoScrollInView
 0001:000007C0       Forms.TScrollingWinControl.CreateWnd
 0001:000007B8       Forms.TScrollingWinControl.Destroy
 0001:000007D8       Forms.TScrollingWinControl.DoGesture
 0001:000007E0       Forms.TScrollingWinControl.DoGetGestureOptions
 0001:000007F0       Forms.TScrollingWinControl.Resizing
 0001:00000770       Graphics.Finalization
 0002:00000088       Graphics.Graphics
 0001:00000758       Graphics.TBrush.SetColor
 0001:00000760       Graphics.TBrush.SetStyle
 0001:00000768       Graphics.TCanvas.SetFont
 0001:00000840       GraphUtil.Finalization
 0002:000000F0       GraphUtil.GraphUtil
 0001:00000828       HelpIntfs.Finalization
 0002:000000D8       HelpIntfs.HelpIntfs
 0001:00002D70       IDEHelp.Finalization
 0002:000001F8       IDEHelp.IDEHelp
 0001:00002CE0       IDEMessages.Finalization
 0002:00000168       IDEMessages.IDEMessages
 0001:00000780       IniFiles.Finalization
 0002:00000098       IniFiles.IniFiles
 0001:00000790       IOUtils.Finalization
 0002:000000A8       IOUtils.IOUtils
 0002:000000A0       IOUtils.TPath.Create@
 0001:00000788       IOUtils.TPath.Destroy@
 0001:00002D58       Mapi.Finalization
 0002:000001E0       Mapi.Mapi
 0001:000007A0       Menus.Finalization
 0002:000000B8       Menus.Menus
 0001:00002CC8       msxmldom.Finalization
 0002:00000150       msxmldom.msxmldom
 0001:000007B0       MultiMon.Finalization
 0002:000000C8       MultiMon.MultiMon
 0001:00002CF8       PercentageDockTree.Finalization
 0002:00000180       PercentageDockTree.PercentageDockTree
 0001:00002D28       PlatformDefaultStyleActnCtrls.Finalization
 0002:000001B0       PlatformDefaultStyleActnCtrls.PlatformDefaultStyleActnCtrls
 0001:000008D0       Printers.Finalization
 0002:00000100       Printers.Printers
 0001:00002D60       Proxies.Finalization
 0002:000001E8       Proxies.Proxies
 0001:00000778       Registry.Finalization
 0002:00000090       Registry.Registry
 0001:00000850       StdCtrls.TCustomGroupBox.AdjustClientRect
 0001:00000848       StdCtrls.TCustomGroupBox.Create
 0001:00000858       StdCtrls.TCustomGroupBox.CreateParams
 0001:00000860       StdCtrls.TCustomGroupBox.Paint
 0001:00002D80       StFilSys.Finalization
 0002:00000208       StFilSys.StFilSys
 0001:00000740       SyncObjs.Finalization
 0002:00000070       SyncObjs.SyncObjs
 0001:00000280       SysInit.@InitPkg
 0001:000002E4       SysInit.@PackageLoad
 0001:000002F0       SysInit.@PackageUnload
 0001:00000170       SysInit.AllocTlsBuffer
 0001:0000022C       SysInit.ExitProcessTLS
 0001:000001F4       SysInit.ExitThreadTLS
 0001:00000138       SysInit.FreeLibrary
 0001:0000017C       SysInit.GetTlsSize
 0004:00000004       SysInit.HInstance
 0001:00000250       SysInit.InitializeModule
 0001:000001C8       SysInit.InitProcessTLS
 0001:00000184       SysInit.InitThreadTLS
 0001:00000140       SysInit.LocalAlloc
 0001:00000148       SysInit.LocalFree
 0003:00000004       SysInit.Module
 0004:00000000       SysInit.ModuleIsLib
 0004:00000001       SysInit.ModuleIsPackage
 0001:00000150       SysInit.TlsAlloc
 0004:00000008       SysInit.tlsBuffer
 0001:00000158       SysInit.TlsFree
 0001:00000160       SysInit.TlsGetValue
 0003:00000000       SysInit.TlsIndex
 0005:00000000       SysInit.TlsLast
 0003:00000020       SysInit.TlsProc
 0001:00000168       SysInit.TlsSetValue
 0001:0000025C       SysInit.UninitializeModule
 0001:00000090       System.@AfterConstruction
 0001:00000098       System.@BeforeDestruction
 0001:00000050       System.@CallDynaInst
 0001:00000080       System.@ClassCreate
 0001:00000088       System.@ClassDestroy
 0001:000000B8       System.@DoneExcept
 0001:000000A0       System.@HandleAnyException
 0001:000000A8       System.@HandleFinally
 0001:000000D8       System.@InitImports
 0001:00000048       System.@IsClass
 0001:000000C8       System.@PackageLoad
 0001:000000D0       System.@PackageUnload
 0001:000000B0       System.@RaiseExcept
 0001:000000E0       System.@RunError
 0001:000000C0       System.@TryFinallyExit
 0001:000000F0       System.@UStrArrayClr
 0001:00000100       System.@UStrCatN
 0001:000000E8       System.@UStrClr
 0001:000000F8       System.@UStrFromString
 0001:00000108       System.AddModuleUnloadProc
 0001:00000130       System.Finalization
 0001:00000128       System.LoadResString
 0001:00000118       System.RegisterModule
 0001:00000110       System.RemoveModuleUnloadProc
 0002:00000000       System.System
 0001:00000070       System.TObject.AfterConstruction
 0001:00000060       System.TObject.ClassInfo
 0001:00000008       System.TObject.ClassName
 0001:00000010       System.TObject.ClassNameIs
 0001:00000018       System.TObject.ClassParent
 0001:00000000       System.TObject.ClassType
 0001:00000078       System.TObject.Dispatch
 0001:00000038       System.TObject.Equals
 0001:00000030       System.TObject.Free
 0001:00000028       System.TObject.FreeInstance
 0001:00000040       System.TObject.GetHashCode
 0001:00000058       System.TObject.InheritsFrom
 0001:00000020       System.TObject.NewInstance
 0001:00000068       System.TObject.ToString
 0001:00000120       System.UnregisterModule
 0001:00000370       SysUtils.Exception.Create
 0002:00000030       SysUtils.Exception.Create@
 0001:00000378       SysUtils.Exception.CreateFmt
 0001:00000380       SysUtils.Exception.Destroy@
 0001:00000398       SysUtils.Finalization
 0002:00000038       SysUtils.SysUtils
 0002:00000028       SysUtils.TEncoding.Create@
 0001:00000390       SysUtils.TEncoding.Destroy@
 0002:00000020       SysUtils.TLanguages.Create@
 0001:00000388       SysUtils.TLanguages.Destroy@
 0001:00002D20       TabDock.Finalization
 0002:000001A8       TabDock.TabDock
 0001:00002D10       Tabs.Finalization
 0002:00000198       Tabs.Tabs
 0001:00000798       Themes.Finalization
 0002:000000B0       Themes.Themes
 0002:00000078       TimeSpan.TTimeSpan.Create@
 0001:00000748       TimeSpan.TTimeSpan.Destroy@
 0001:00002CB0       ToolsAPI.Finalization
 0002:00000138       ToolsAPI.ToolsAPI
 0001:00002D90       TopLevels.Finalization
 0002:00000218       TopLevels.TopLevels
 0001:00002D98       TreeIntf.Finalization
 0002:00000220       TreeIntf.TreeIntf
 0001:00000450       TypInfo.Finalization
 0001:00000448       TypInfo.GetTypeData
 0002:00000050       TypInfo.TypInfo
 0001:000007A8       UxTheme.Finalization
 0002:000000C0       UxTheme.UxTheme
 0001:00000458       Variants.Finalization
 0002:00000058       Variants.Variants
 0001:00000460       VarUtils.Finalization
 0002:00000060       VarUtils.VarUtils
 0001:00002CA0       VCLEditors.Finalization
 0002:00000120       VCLEditors.TActionResourceCache.Create@
 0001:00002C98       VCLEditors.TActionResourceCache.Destroy@
 0002:00000128       VCLEditors.VCLEditors
 0001:00002D88       WideStrings.Finalization
 0002:00000210       WideStrings.WideStrings
 0004:0000000C       Windows..2
 0001:00000350       Windows.Finalization
 0001:000002FC       Windows.FreeLibrary
 0001:00000304       Windows.GetVersionEx
 0004:00000010       Windows.HtmlHelpModule
 0001:00000314       Windows.InitVersionInfo
 0001:0000030C       Windows.VirtualQuery
 0003:00000030       Windows.Win32MajorVersion
 0003:00000034       Windows.Win32MinorVersion
 0003:00000038       Windows.Win32Platform
 0002:00000008       Windows.Windows
 0001:00002CC0       xmldom.Finalization
 0002:00000148       xmldom.xmldom
 0001:00002CB8       XMLIntf.Finalization
 0002:00000140       XMLIntf.XMLIntf


  Address             Publics by Value

 0001:00000000       System.TObject.ClassType
 0001:00000008       System.TObject.ClassName
 0001:00000010       System.TObject.ClassNameIs
 0001:00000018       System.TObject.ClassParent
 0001:00000020       System.TObject.NewInstance
 0001:00000028       System.TObject.FreeInstance
 0001:00000030       System.TObject.Free
 0001:00000038       System.TObject.Equals
 0001:00000040       System.TObject.GetHashCode
 0001:00000048       System.@IsClass
 0001:00000050       System.@CallDynaInst
 0001:00000058       System.TObject.InheritsFrom
 0001:00000060       System.TObject.ClassInfo
 0001:00000068       System.TObject.ToString
 0001:00000070       System.TObject.AfterConstruction
 0001:00000078       System.TObject.Dispatch
 0001:00000080       System.@ClassCreate
 0001:00000088       System.@ClassDestroy
 0001:00000090       System.@AfterConstruction
 0001:00000098       System.@BeforeDestruction
 0001:000000A0       System.@HandleAnyException
 0001:000000A8       System.@HandleFinally
 0001:000000B0       System.@RaiseExcept
 0001:000000B8       System.@DoneExcept
 0001:000000C0       System.@TryFinallyExit
 0001:000000C8       System.@PackageLoad
 0001:000000D0       System.@PackageUnload
 0001:000000D8       System.@InitImports
 0001:000000E0       System.@RunError
 0001:000000E8       System.@UStrClr
 0001:000000F0       System.@UStrArrayClr
 0001:000000F8       System.@UStrFromString
 0001:00000100       System.@UStrCatN
 0001:00000108       System.AddModuleUnloadProc
 0001:00000110       System.RemoveModuleUnloadProc
 0001:00000118       System.RegisterModule
 0001:00000120       System.UnregisterModule
 0001:00000128       System.LoadResString
 0001:00000130       System.Finalization
 0001:00000138       SysInit.FreeLibrary
 0001:00000140       SysInit.LocalAlloc
 0001:00000148       SysInit.LocalFree
 0001:00000150       SysInit.TlsAlloc
 0001:00000158       SysInit.TlsFree
 0001:00000160       SysInit.TlsGetValue
 0001:00000168       SysInit.TlsSetValue
 0001:00000170       SysInit.AllocTlsBuffer
 0001:0000017C       SysInit.GetTlsSize
 0001:00000184       SysInit.InitThreadTLS
 0001:000001C8       SysInit.InitProcessTLS
 0001:000001F4       SysInit.ExitThreadTLS
 0001:0000022C       SysInit.ExitProcessTLS
 0001:00000250       SysInit.InitializeModule
 0001:0000025C       SysInit.UninitializeModule
 0001:00000280       SysInit.@InitPkg
 0001:000002E4       SysInit.@PackageLoad
 0001:000002F0       SysInit.@PackageUnload
 0001:000002FC       Windows.FreeLibrary
 0001:00000304       Windows.GetVersionEx
 0001:0000030C       Windows.VirtualQuery
 0001:00000314       Windows.InitVersionInfo
 0001:00000350       Windows.Finalization
 0001:00000370       SysUtils.Exception.Create
 0001:00000378       SysUtils.Exception.CreateFmt
 0001:00000380       SysUtils.Exception.Destroy@
 0001:00000388       SysUtils.TLanguages.Destroy@
 0001:00000390       SysUtils.TEncoding.Destroy@
 0001:00000398       SysUtils.Finalization
 0001:000003A0       Classes.InitInheritedComponent
 0001:000003A8       Classes.TList.Add
 0001:000003B0       Classes.TList.Delete
 0001:000003B8       Classes.TList.Get
 0001:000003C0       Classes.TThreadList.Create
 0001:000003C8       Classes.TThreadList.LockList
 0001:000003D0       Classes.TThreadList.Remove
 0001:000003D8       Classes.TThreadList.UnlockList
 0001:000003E0       Classes.TPersistent.Assign
 0001:000003E8       Classes.TThread.Destroy@
 0001:000003F0       Classes.TComponent.BeforeDestruction
 0001:000003F8       Classes.TComponent.WriteState
 0001:00000400       Classes.TComponent.ValidateRename
 0001:00000408       Classes.TComponent.GetComponent
 0001:00000410       Classes.TComponent.GetComponentCount
 0001:00000418       Classes.TComponent.SetComponentIndex
 0001:00000420       Classes.TComponent.UpdateAction
 0001:00000428       Classes.TComponent.SafeCallException
 0001:00000430       Classes.TComponent.UpdateRegistry
 0001:00000438       Classes.TComponent.QueryInterface
 0001:00000440       Classes.Finalization
 0001:00000448       TypInfo.GetTypeData
 0001:00000450       TypInfo.Finalization
 0001:00000458       Variants.Finalization
 0001:00000460       VarUtils.Finalization
 0001:00000468       DesignIntf.RegisterCustomModule
 0001:00000470       Controls.TControl.GetDragImages
 0001:00000478       Controls.TControl.GetEnabled
 0001:00000480       Controls.TControl.GetAction
 0001:00000488       Controls.TControl.SetAnchors
 0001:00000490       Controls.TControl.IsAnchorsStored
 0001:00000498       Controls.TControl.SetDragMode
 0001:000004A0       Controls.TControl.GetDragMode
 0001:000004A8       Controls.TControl.SetAlign
 0001:000004B0       Controls.TControl.SetWidth
 0001:000004B8       Controls.TControl.SetHeight
 0001:000004C0       Controls.TControl.SetAutoSize
 0001:000004C8       Controls.TControl.SetName
 0001:000004D0       Controls.TControl.SetVisible
 0001:000004D8       Controls.TControl.SetEnabled
 0001:000004E0       Controls.TControl.SetPopupMenu
 0001:000004E8       Controls.TControl.GetText
 0001:000004F0       Controls.TControl.SetText
 0001:000004F8       Controls.TControl.SetBiDiMode
 0001:00000500       Controls.TControl.SetFont
 0001:00000508       Controls.TControl.IsFontStored
 0001:00000510       Controls.TControl.IsShowHintStored
 0001:00000518       Controls.TControl.IsBiDiModeStored
 0001:00000520       Controls.TControl.SetParentFont
 0001:00000528       Controls.TControl.SetShowHint
 0001:00000530       Controls.TControl.SetParentShowHint
 0001:00000538       Controls.TControl.SetColor
 0001:00000540       Controls.TControl.IsColorStored
 0001:00000548       Controls.TControl.SetParentColor
 0001:00000550       Controls.TControl.SetParentBiDiMode
 0001:00000558       Controls.TControl.DoGesture
 0001:00000560       Controls.TControl.DoGetGestureOptions
 0001:00000568       Controls.TControl.CreateTouchManager
 0001:00000570       Controls.TControl.IsCaptionStored
 0001:00000578       Controls.TControl.IsEnabledStored
 0001:00000580       Controls.TControl.IsVisibleStored
 0001:00000588       Controls.TControl.IsOnClickStored
 0001:00000590       Controls.TControl.Loaded
 0001:00000598       Controls.TControl.GetFloating
 0001:000005A0       Controls.TControl.GetFloatingDockSiteClass
 0001:000005A8       Controls.TControl.InitiateAction
 0001:000005B0       Controls.TControl.SetConstraints
 0001:000005B8       Controls.TWinControl.ReadState
 0001:000005C0       Controls.TWinControl.AlignControls
 0001:000005C8       Controls.TWinControl.GetControlCount
 0001:000005D0       Controls.TWinControl.Notification
 0001:000005D8       Controls.TWinControl.CreateWnd
 0001:000005E0       Controls.TWinControl.CreateWindowHandle
 0001:000005E8       Controls.TWinControl.DefineProperties
 0001:000005F0       Controls.TWinControl.DestroyWnd
 0001:000005F8       Controls.TWinControl.DestroyWindowHandle
 0001:00000600       Controls.TWinControl.CreateHandle
 0001:00000608       Controls.TWinControl.CustomAlignInsertBefore
 0001:00000610       Controls.TWinControl.CustomAlignPosition
 0001:00000618       Controls.TWinControl.DestroyHandle
 0001:00000620       Controls.TWinControl.SetParentDoubleBuffered
 0001:00000628       Controls.TWinControl.WndProc
 0001:00000630       Controls.TWinControl.DefaultHandler
 0001:00000638       Controls.TWinControl.RequestAlign
 0001:00000640       Controls.TWinControl.SetDockSite
 0001:00000648       Controls.TWinControl.SetBounds
 0001:00000650       Controls.TWinControl.ShowControl
 0001:00000658       Controls.TWinControl.GetDeviceContext
 0001:00000660       Controls.TWinControl.Invalidate
 0001:00000668       Controls.TWinControl.Update
 0001:00000670       Controls.TWinControl.Repaint
 0001:00000678       Controls.TWinControl.SetFocus
 0001:00000680       Controls.TWinControl.GetControlExtents
 0001:00000688       Controls.TWinControl.GetClientOrigin
 0001:00000690       Controls.TWinControl.GetClientRect
 0001:00000698       Controls.TWinControl.SetCtl3D
 0001:000006A0       Controls.TWinControl.IsCtl3DStored
 0001:000006A8       Controls.TWinControl.SetParentCtl3D
 0001:000006B0       Controls.TWinControl.GetTabOrder
 0001:000006B8       Controls.TWinControl.SetTabOrder
 0001:000006C0       Controls.TWinControl.SetTabStop
 0001:000006C8       Controls.TWinControl.SetUseDockManager
 0001:000006D0       Controls.TWinControl.HandleAllocated
 0001:000006D8       Controls.TWinControl.GetChildren
 0001:000006E0       Controls.TWinControl.SetChildOrder
 0001:000006E8       Controls.TWinControl.CanResize
 0001:000006F0       Controls.TWinControl.ConstrainedResize
 0001:000006F8       Controls.TWinControl.AssignTo
 0001:00000700       Controls.TWinControl.CanAutoSize
 0001:00000708       Controls.TWinControl.SetParentBackground
 0001:00000710       Controls.TWinControl.DockReplaceDockClient
 0001:00000718       Controls.TWinControl.UpdateControlOriginalParentSize
 0001:00000720       Controls.TWinControl.SetParent
 0001:00000728       Controls.TCustomControl.Destroy
 0001:00000730       Controls.TCustomControl.PaintWindow
 0001:00000738       Controls.Finalization
 0001:00000740       SyncObjs.Finalization
 0001:00000748       TimeSpan.TTimeSpan.Destroy@
 0001:00000750       ActnList.Finalization
 0001:00000758       Graphics.TBrush.SetColor
 0001:00000760       Graphics.TBrush.SetStyle
 0001:00000768       Graphics.TCanvas.SetFont
 0001:00000770       Graphics.Finalization
 0001:00000778       Registry.Finalization
 0001:00000780       IniFiles.Finalization
 0001:00000788       IOUtils.TPath.Destroy@
 0001:00000790       IOUtils.Finalization
 0001:00000798       Themes.Finalization
 0001:000007A0       Menus.Finalization
 0001:000007A8       UxTheme.Finalization
 0001:000007B0       MultiMon.Finalization
 0001:000007B8       Forms.TScrollingWinControl.Destroy
 0001:000007C0       Forms.TScrollingWinControl.CreateWnd
 0001:000007C8       Forms.TScrollingWinControl.AlignControls
 0001:000007D0       Forms.TScrollingWinControl.AutoScrollEnabled
 0001:000007D8       Forms.TScrollingWinControl.DoGesture
 0001:000007E0       Forms.TScrollingWinControl.DoGetGestureOptions
 0001:000007E8       Forms.TScrollingWinControl.AutoScrollInView
 0001:000007F0       Forms.TScrollingWinControl.Resizing
 0001:000007F8       Forms.TScrollingWinControl.AdjustClientRect
 0001:00000800       Forms.TScrollBox.Create
 0001:00000808       Forms.TScrollBox.CreateParams
 0001:00000810       Forms.TScrollBox.PaintWindow
 0001:00000818       Forms.TApplication.HandleException
 0001:00000820       Forms.Finalization
 0001:00000828       HelpIntfs.Finalization
 0001:00000830       Dialogs.Finalization
 0001:00000838       ComCtrls.Finalization
 0001:00000840       GraphUtil.Finalization
 0001:00000848       StdCtrls.TCustomGroupBox.Create
 0001:00000850       StdCtrls.TCustomGroupBox.AdjustClientRect
 0001:00000858       StdCtrls.TCustomGroupBox.CreateParams
 0001:00000860       StdCtrls.TCustomGroupBox.Paint
 0001:00000868       ExtCtrls.Frame3D
 0001:00000870       ExtCtrls.TCustomPanel.Create
 0001:00000878       ExtCtrls.TCustomPanel.CreateParams
 0001:00000880       ExtCtrls.TCustomPanel.SetAlignment
 0001:00000888       ExtCtrls.TCustomPanel.SetBevelInner
 0001:00000890       ExtCtrls.TCustomPanel.SetBevelOuter
 0001:00000898       ExtCtrls.TCustomPanel.SetBevelWidth
 0001:000008A0       ExtCtrls.TCustomPanel.SetBorderWidth
 0001:000008A8       ExtCtrls.TCustomPanel.SetBorderStyle
 0001:000008B0       ExtCtrls.TCustomPanel.AdjustClientRect
 0001:000008B8       ExtCtrls.TCustomPanel.CanAutoSize
 0001:000008C0       ExtCtrls.TCustomPanel.SetParentBackground
 0001:000008C8       ExtCtrls.Finalization
 0001:000008D0       Printers.Finalization
 0001:000008D8       Clipbrd.Finalization
 0001:000008E0       FlatSB.Finalization
 0001:000008E8       Boxes..TBox
 0001:000014C0       Boxes..TControlGroupBox
 0001:00001F20       Boxes..TControlScrollBox
 0001:000021C0       Boxes.TBox.Create
 0001:00002328       Boxes.TBox.Destroy
 0001:000023B0       Boxes.TBox.CreateParams
 0001:000023D8       Boxes.TBox.SetParent
 0001:00002408       Boxes.AdjustColors
 0001:00002440       Boxes.TBox.Paint
 0001:00002500       Boxes.TBox.GetChildren
 0001:0000256C       Boxes.TBox.SetChildOrder
 0001:00002600       Boxes.TControlGroupBox.Create
 0001:00002768       Boxes.TControlGroupBox.Destroy
 0001:000027F0       Boxes.TControlGroupBox.CreateParams
 0001:00002818       Boxes.TControlGroupBox.SetParent
 0001:00002848       Boxes.TControlGroupBox.GetChildren
 0001:000028B4       Boxes.TControlGroupBox.SetChildOrder
 0001:00002948       Boxes.TControlScrollBox.Create
 0001:00002AB0       Boxes.TControlScrollBox.Destroy
 0001:00002B38       Boxes.TControlScrollBox.CreateParams
 0001:00002B60       Boxes.TControlScrollBox.SetParent
 0001:00002B90       Boxes.TControlScrollBox.GetChildren
 0001:00002BFC       Boxes.TControlScrollBox.SetChildOrder
 0001:00002C90       Boxes.Finalization
 0001:00002C98       VCLEditors.TActionResourceCache.Destroy@
 0001:00002CA0       VCLEditors.Finalization
 0001:00002CA8       DesignEditors.Finalization
 0001:00002CB0       ToolsAPI.Finalization
 0001:00002CB8       XMLIntf.Finalization
 0001:00002CC0       xmldom.Finalization
 0001:00002CC8       msxmldom.Finalization
 0001:00002CD0       ComObj.Finalization
 0001:00002CD8       DockForm.Finalization
 0001:00002CE0       IDEMessages.Finalization
 0001:00002CE8       DeskForm.Finalization
 0001:00002CF0       BaseDock.Finalization
 0001:00002CF8       PercentageDockTree.Finalization
 0001:00002D00       CaptionedDockTree.Finalization
 0001:00002D08       DockTabSet.Finalization
 0001:00002D10       Tabs.Finalization
 0001:00002D18       DeskUtil.Finalization
 0001:00002D20       TabDock.Finalization
 0001:00002D28       PlatformDefaultStyleActnCtrls.Finalization
 0001:00002D30       Buttons.Finalization
 0001:00002D38       ActnMan.Finalization
 0001:00002D40       ActnMenus.Finalization
 0001:00002D48       ExtActns.Finalization
 0001:00002D50       ExtDlgs.Finalization
 0001:00002D58       Mapi.Finalization
 0001:00002D60       Proxies.Finalization
 0001:00002D68       ComponentDesigner.Finalization
 0001:00002D70       IDEHelp.Finalization
 0001:00002D78       AxCtrls.Finalization
 0001:00002D80       StFilSys.Finalization
 0001:00002D88       WideStrings.Finalization
 0001:00002D90       TopLevels.Finalization
 0001:00002D98       TreeIntf.Finalization
 0001:00002DA0       AppEvnts.Finalization
 0001:00002DE8       ccreg.IsBaseContainer
 0001:00002E08       ccreg.GetBaseContainer
 0001:00002E3C       ccreg.ClassNotFound
 0001:00002EA8       ccreg.GetCustomContainerClass
 0001:00002F30       ccreg.FindCustomContainerClass
 0001:00002F50       ccreg.GetCustomContainerUnit
 0001:00002F74       ccreg.GetCustomContainerClass
 0001:00002FCC       ccreg.GetCustomContainerClassListCount
 0001:00003014       ccreg.RegisterCustomContainer
 0001:00003128       ccreg.UnRegisterCustomContainer
 0001:00003138       ccreg.UnRegisterCustomContainerClasses
 0001:000031BC       ccreg.ModuleUnload
 0001:00003210       ccreg.Finalization
 0001:00003238       ccregprc.RegisterCustomContainerProcImpl
 0001:00003464       ccregprc.InitBaseContainerList
 0001:00003484       ccregprc.Finalization
 0001:00003998       .ccpackD2010.@GetPackageInfoTable
 0001:000039A0       .ccpackD2010.@PackageLoad
 0001:000039AC       .ccpackD2010.@PackageUnload
 0002:00000000       System.System
 0002:00000008       Windows.Windows
 0002:00000020       SysUtils.TLanguages.Create@
 0002:00000028       SysUtils.TEncoding.Create@
 0002:00000030       SysUtils.Exception.Create@
 0002:00000038       SysUtils.SysUtils
 0002:00000040       Classes.TThread.Create@
 0002:00000048       Classes.Classes
 0002:00000050       TypInfo.TypInfo
 0002:00000058       Variants.Variants
 0002:00000060       VarUtils.VarUtils
 0002:00000068       Controls.Controls
 0002:00000070       SyncObjs.SyncObjs
 0002:00000078       TimeSpan.TTimeSpan.Create@
 0002:00000080       ActnList.ActnList
 0002:00000088       Graphics.Graphics
 0002:00000090       Registry.Registry
 0002:00000098       IniFiles.IniFiles
 0002:000000A0       IOUtils.TPath.Create@
 0002:000000A8       IOUtils.IOUtils
 0002:000000B0       Themes.Themes
 0002:000000B8       Menus.Menus
 0002:000000C0       UxTheme.UxTheme
 0002:000000C8       MultiMon.MultiMon
 0002:000000D0       Forms.Forms
 0002:000000D8       HelpIntfs.HelpIntfs
 0002:000000E0       Dialogs.Dialogs
 0002:000000E8       ComCtrls.ComCtrls
 0002:000000F0       GraphUtil.GraphUtil
 0002:000000F8       ExtCtrls.ExtCtrls
 0002:00000100       Printers.Printers
 0002:00000108       Clipbrd.Clipbrd
 0002:00000110       FlatSB.FlatSB
 0002:00000118       Boxes.Boxes
 0002:00000120       VCLEditors.TActionResourceCache.Create@
 0002:00000128       VCLEditors.VCLEditors
 0002:00000130       DesignEditors.DesignEditors
 0002:00000138       ToolsAPI.ToolsAPI
 0002:00000140       XMLIntf.XMLIntf
 0002:00000148       xmldom.xmldom
 0002:00000150       msxmldom.msxmldom
 0002:00000158       ComObj.ComObj
 0002:00000160       DockForm.DockForm
 0002:00000168       IDEMessages.IDEMessages
 0002:00000170       DeskForm.DeskForm
 0002:00000178       BaseDock.BaseDock
 0002:00000180       PercentageDockTree.PercentageDockTree
 0002:00000188       CaptionedDockTree.CaptionedDockTree
 0002:00000190       DockTabSet.DockTabSet
 0002:00000198       Tabs.Tabs
 0002:000001A0       DeskUtil.DeskUtil
 0002:000001A8       TabDock.TabDock
 0002:000001B0       PlatformDefaultStyleActnCtrls.PlatformDefaultStyleActnCtrls
 0002:000001B8       Buttons.Buttons
 0002:000001C0       ActnMan.ActnMan
 0002:000001C8       ActnMenus.ActnMenus
 0002:000001D0       ExtActns.ExtActns
 0002:000001D8       ExtDlgs.ExtDlgs
 0002:000001E0       Mapi.Mapi
 0002:000001E8       Proxies.Proxies
 0002:000001F0       ComponentDesigner.ComponentDesigner
 0002:000001F8       IDEHelp.IDEHelp
 0002:00000200       AxCtrls.AxCtrls
 0002:00000208       StFilSys.StFilSys
 0002:00000210       WideStrings.WideStrings
 0002:00000218       TopLevels.TopLevels
 0002:00000220       TreeIntf.TreeIntf
 0002:00000228       AppEvnts.AppEvnts
 0002:00000230       ccreg.ccreg
 0002:00000260       ccregprc.ccregprc
 0002:0000027C       .ccpackD2010..ccpackD2010
 0003:00000000       SysInit.TlsIndex
 0003:00000004       SysInit.Module
 0003:00000020       SysInit.TlsProc
 0003:00000030       Windows.Win32MajorVersion
 0003:00000034       Windows.Win32MinorVersion
 0003:00000038       Windows.Win32Platform
 0003:0000003C       ccreg.RegisterCustomContainerProc
 0003:00000040       ccreg.BaseContainerClassArray
 0003:00000058       ccreg.CustomContainerClassList
 0004:00000000       SysInit.ModuleIsLib
 0004:00000001       SysInit.ModuleIsPackage
 0004:00000004       SysInit.HInstance
 0004:00000008       SysInit.tlsBuffer
 0004:0000000C       Windows..2
 0004:00000010       Windows.HtmlHelpModule
 0004:00000014       Boxes..4
 0004:00000018       ccreg..1
 0004:0000001C       ccregprc..1
 0005:00000000       SysInit.TlsLast


Line numbers for Boxes(Boxes.pas) segment .text

   199 0001:000021C0   200 0001:000021F1   201 0001:000021FB   203 0001:0000221C
   204 0001:00002237   205 0001:00002275   206 0001:00002282   207 0001:00002290
   209 0001:000022B1   214 0001:000022C7   215 0001:000022D4   217 0001:000022E1
   220 0001:00002328   221 0001:0000233C   222 0001:00002349   223 0001:00002357
   225 0001:00002378   227 0001:0000238C   228 0001:0000239B   231 0001:000023B0
   232 0001:000023B6   233 0001:000023BF   234 0001:000023C5   235 0001:000023D5
   238 0001:000023D8   239 0001:000023DE   240 0001:000023EF   241 0001:000023F9
   242 0001:00002402   252 0001:00002408   253 0001:0000240B   254 0001:00002415
   255 0001:00002423   256 0001:0000242D   257 0001:0000243B   259 0001:00002440
   260 0001:0000244A   261 0001:00002454   263 0001:0000245F   264 0001:00002466
   266 0001:00002482   267 0001:0000249D   269 0001:000024A8   270 0001:000024AF
   272 0001:000024CB   274 0001:000024D1   275 0001:000024DC   276 0001:000024E6
   277 0001:000024F0   279 0001:000024FA   285 0001:00002500   286 0001:0000250D
   287 0001:0000251C   288 0001:00002520   290 0001:00002537   291 0001:00002543
   292 0001:0000255A   288 0001:0000255D   293 0001:00002562   298 0001:0000256C
   299 0001:0000257C   300 0001:0000258E   303 0001:0000259E   304 0001:000025A9
   305 0001:000025B1   306 0001:000025C2   308 0001:000025D8   309 0001:000025DC
   311 0001:000025E6   312 0001:000025F0   314 0001:000025F2   305 0001:000025F3
   316 0001:000025F6   321 0001:00002600   322 0001:00002631   323 0001:0000263B
   325 0001:0000265C   326 0001:00002677   327 0001:000026B5   328 0001:000026C2
   329 0001:000026D0   331 0001:000026F1   336 0001:00002707   337 0001:00002714
   339 0001:00002721   342 0001:00002768   343 0001:0000277C   344 0001:00002789
   345 0001:00002797   347 0001:000027B8   349 0001:000027CC   350 0001:000027DB
   353 0001:000027F0   354 0001:000027F6   355 0001:000027FF   356 0001:00002805
   357 0001:00002815   360 0001:00002818   361 0001:0000281E   362 0001:0000282F
   363 0001:00002839   364 0001:00002842   370 0001:00002848   371 0001:00002855
   372 0001:00002864   373 0001:00002868   375 0001:0000287F   376 0001:0000288B
   377 0001:000028A2   373 0001:000028A5   378 0001:000028AA   383 0001:000028B4
   384 0001:000028C4   385 0001:000028D6   388 0001:000028E6   389 0001:000028F1
   390 0001:000028F9   391 0001:0000290A   393 0001:00002920   394 0001:00002924
   396 0001:0000292E   397 0001:00002938   399 0001:0000293A   390 0001:0000293B
   401 0001:0000293E   406 0001:00002948   407 0001:00002979   408 0001:00002983
   410 0001:000029A4   411 0001:000029BF   412 0001:000029FD   413 0001:00002A0A
   414 0001:00002A18   416 0001:00002A39   421 0001:00002A4F   422 0001:00002A5C
   424 0001:00002A69   427 0001:00002AB0   428 0001:00002AC4   429 0001:00002AD1
   430 0001:00002ADF   432 0001:00002B00   434 0001:00002B14   435 0001:00002B23
   438 0001:00002B38   439 0001:00002B3E   440 0001:00002B47   441 0001:00002B4D
   442 0001:00002B5D   445 0001:00002B60   446 0001:00002B66   447 0001:00002B77
   448 0001:00002B81   449 0001:00002B8A   455 0001:00002B90   456 0001:00002B9D
   457 0001:00002BAC   458 0001:00002BB0   460 0001:00002BC7   461 0001:00002BD3
   462 0001:00002BEA   458 0001:00002BED   463 0001:00002BF2   468 0001:00002BFC
   469 0001:00002C0C   470 0001:00002C1E   473 0001:00002C2E   474 0001:00002C39
   475 0001:00002C41   476 0001:00002C52   478 0001:00002C68   479 0001:00002C6C
   481 0001:00002C76   482 0001:00002C80   484 0001:00002C82   475 0001:00002C83
   486 0001:00002C86

Line numbers for Boxes(Boxes.pas) segment .itext

   488 0002:00000118

Line numbers for ccreg(ccreg.pas) segment .text

    67 0001:00002DE8    68 0001:00002DE9    69 0001:00002DEC    70 0001:00002DF3
    72 0001:00002DF7    73 0001:00002DF9    74 0001:00002DFB    69 0001:00002DFF
    75 0001:00002E04    80 0001:00002E08    81 0001:00002E0E    82 0001:00002E11
    83 0001:00002E18    85 0001:00002E25    86 0001:00002E27    87 0001:00002E29
    82 0001:00002E2D    88 0001:00002E32    91 0001:00002E3C    92 0001:00002E58
    93 0001:00002E86    98 0001:00002EA8    99 0001:00002EB4   100 0001:00002EC0
   101 0001:00002ECE   103 0001:00002ED9   104 0001:00002EE5   105 0001:00002EFB
   101 0001:00002EFC   106 0001:00002EFF   108 0001:00002F11   110 0001:00002F23
   113 0001:00002F30   114 0001:00002F34   115 0001:00002F3D   116 0001:00002F48
   119 0001:00002F50   120 0001:00002F56   121 0001:00002F71   124 0001:00002F74
   125 0001:00002F7C   126 0001:00002F88   127 0001:00002F96   129 0001:00002FAF
   131 0001:00002FC1   134 0001:00002FCC   135 0001:00002FD0   136 0001:00002FDA
   137 0001:00002FE8   139 0001:00002FFB   141 0001:0000300D   165 0001:00003014
   166 0001:0000302C   167 0001:00003035   169 0001:0000303F   170 0001:00003077
   171 0001:00003081   172 0001:0000308F   174 0001:000030A3   176 0001:000030B5
   180 0001:00003128   181 0001:00003134   187 0001:00003138   188 0001:00003143
   189 0001:0000314F   190 0001:0000315D   192 0001:00003166   193 0001:0000317B
   194 0001:00003184   195 0001:0000318D   190 0001:0000318E   197 0001:000031A0
   199 0001:000031B2   203 0001:000031BC   204 0001:000031C1   210 0001:00003210
   211 0001:00003222   212 0001:0000322C   213 0001:00003236

Line numbers for ccreg(ccreg.pas) segment .itext

   206 0002:00000230   207 0002:00000243   208 0002:0000024D   209 0002:0000025E

Line numbers for ccregprc(ccregprc.pas) segment .text

    40 0001:00003238    41 0001:00003250    42 0001:0000325A    44 0001:00003292
    45 0001:000032B3    47 0001:000032C5    49 0001:000032E6    51 0001:000032F5
    56 0001:00003349    57 0001:00003356    62 0001:00003464    63 0001:00003466
    64 0001:00003471    63 0001:0000347B    65 0001:0000347E    71 0001:00003484
    72 0001:00003495

Line numbers for ccregprc(ccregprc.pas) segment .itext

    67 0002:00000260    68 0002:00000269    69 0002:00000274    70 0002:00000279

Line numbers for .ccpackD2010(ccpackD2010.dpk) segment .itext

    38 0002:0000027C

Bound resource files

ccpackD2010.res
ccpackD2010.drf


Program entry point at 0002:0000027C
